:1000000041C0AFC1A0C1B0C1AFC1AEC199C11FC194
:10001000ABC1AAC1A9C1A8C1A7C1763431F101639E
:100020002200FA22B9AB63CBDBA2FBEB64003C00FD
:1000300028001400140100D9133BD85B11005BF3B6
:100040005900010101012999C398299BC39A089578
:100050002999C39A299BC3980895289B9098289919
:10006000909A0895289B909A289990980895C49AF8
:100070000895C49808950370F02E08B30C7F0F29DB
:1000800008BB08956624DD27FF2702E00EBF0FE5B9
:100090000DBF0FE168BA07BB01E201BB00E002BB84
:1000A000E1DF00E006B907E007B900EC0BBF0BE0A9
:1000B00005BF03E003BF02E809BF0FEF02BF01E283
:1000C0000FBD01E00EBD68BC7724442708E101BDE7
:1000D0000AE101BD789480D1FBD2B3FCFED200913D
:1000E0008900001F00938B0001E000936600002749
:1000F0000093670001E00093680000936900A5D0B9
:1001000000E008BD08E2D62CE02E66D160927000B7
:100110006092800053D297D1BB20F1F7AADF98DF1D
:1001200000E0A9DF1127139505E0B0FE02C0C6E686
:1001300009C01127B1FE02C0C7E604C0B2FE09C063
:10014000C8E602E0F880F394F01608F0F12EF88289
:10015000DDCFC9E6B3FE04C00EE111E0BDD1DBCFB7
:10016000B4FE04C001E01FEFB7D1D5CFB5FC03C08A
:10017000D9CF442757C097D205E0E0160CF4E02E03
:10018000C9E60991099300E0099304E0088316D2B7
:10019000AA24FF2700916700002309F00395039527
:1001A000302F00916600102F002309F43FEF0A95CD
:1001B000363009F460DF07E0100FCBD2902E789430
:1001C000BB20F1F7E2E4D3D1363019F441DF4FDF41
:1001D00002C04FDF38DFA8ECB0E0B7FFFECF432FFF
:1001E000CBE608810A950F3F39F4CA9508810A9534
:1001F00009930F3FB9F00BE30883CA9540D1A8EEED
:10020000B3E0B6FC0FC0B7FFFCCF0091680000233D
:1002100039F700916B00027019F44F3F01F3E0CF02
:100220004FEFDECF4FEF08E2D62CE02EE6E3B6FE2E
:10023000AED1A4E6B0E0B7FFFECF609270004427D5
:10024000A4E6B0E0B7FFFECF61CF22D208954FB64B
:100250000F930FEF02BF8A9499F409E1802E539512
:100260004423E9F04530C1F14630E9F04F3F71F1E8
:100270005B3431F443955FE5959860927000A895E2
:1002800074D05A9449F40DE7502E772009F07A94EF
:1002900051D0B7FF119770D00F914FBE1895E2DE85
:1002A0009598A895EDCF00916600002341F000914C
:1002B0007000869B0064879B006200937000513041
:1002C00019F4CBDE60927000A895DACFCBDE95985A
:1002D000A89560927000D4CF959B05C0C394C914B3
:1002E00011F49598A895593119F4CC24959AC8CF52
:1002F000563419F49598A895C3CF5B3411F4ADDE4C
:10030000BFCF5C3411F4AEDEBBCF5B3490F05F3511
:1003100064F400916600002341F000917000869B18
:100320000064879B0062009370005A3509F0A8CFE3
:10033000432FA6CFEE2019F0DA9409F4EA94089539
:100340004FB60F93A9CF4FB60F935A3548F0562D9D
:1003500000917000009380006092700001E0802E98
:100360009BCF4FB60F9398CFFFCF772011F0C29A53
:100370000895C298089508950FEF6ABA0BBB63956C
:10038000770F663010F0662771E000E404BBCF936E
:10039000C0E6C60F0881C9B36BBA74BB0ABBC0956F
:1003A00000917400C01729F0C093740000E5009319
:1003B0007300009173000A9519F40395B0907400CE
:1003C0000093730000916500C09180000F710C2BA9
:1003D00000936500CF91089506E001C004E0C0E6F7
:1003E00069920A95E9F708950395FF240894FF1C84
:1003F0000A95E9F70F2D0895102F0F70065F105121
:10040000E8F70A500895FF240A5010F0F394FCCF47
:10041000065F0895F8DFFF0CFF0CFF0CFF0C0F299F
:100420000895F1DF02D0102F0F2DEF93E2E2E00FDD
:10043000C895002DEF91089500918C00D5DF0093B1
:100440006400088112C000916700CEDF0093650050
:1004500000916600C9DF102F009168000B5FC4DFB8
:10046000012B009364000091690060926300609228
:100470006200D7DF00936100109360000895099136
:10048000D0DF00936300109362000991CADFF990F6
:100490000F291F2900936100109360000895F22C2A
:1004A0000881031521F0010D0883FA94C9F7F214AD
:1004B000089500D0A82FBB27BB208894C9F3B7FFAD
:1004C000FBCF08940895EBDF08F478D0CEDFF1DF9E
:1004D00078F79A95C1F70895112E302E8FEF91E09D
:1004E000292EF1DF60F48EE695E0EDDF40F49CE02C
:1004F00080E5E9DF20F49AE08DE2E5DFE0F308959E
:10050000F22C0881010D07FF02C0032D0A95031587
:1005100009F400270883FA94A1F7089500D0A82FC2
:10052000BB27BB208894C9F3B7FFFBCF089408957D
:10053000E7DF44D0CF93CDE6A2DFCF91EFDF68F7BE
:100540009A95B1F70895112E302E8FEF91E0292E54
:10055000EFDF60F48EE695E0EBDF40F49CE080E5B1
:10056000E7DF20F49AE08DE2E3DFE0F30895C89539
:1005700000926300E395C89500926200E395C895E8
:1005800000926100E395C895009260000895EFDF46
:1005900010E11F930FEF702EA8EEB3E0BB2011F413
:1005A000B7FFFCCF1F91BB2041F41A9591F7AFEF35
:1005B000BFE7BB2011F4B7FFFCCF08950F9309E10B
:1005C000702E0F91089520E12A95F1F7089528E003
:1005D0002A95F1F708958E9A8F98F5DF8E98F7DFB8
:1005E000082F8F9AF4DF0894001F01C0000F59F004
:1005F0008E9A18F400008F9802C08F9A00C0E3DF33
:100600008E98E1DFF3CF8E9A8F98DDDF8E98869BF0
:10061000FECF889487990894D6DF089580FFE3CFB2
:10062000991F01E08E9ACFDF8E98CDDF889487994D
:100630000894001FB8F78E9A979510F48F9801C010
:100640008F9AC1DF8E98869BFECFBDDF08958E9A6C
:100650008F9AB9DF8E98BBDF8F98B5DF0895969893
:1006600097988E988F98089580EDBADF0F2DD6DF7A
:10067000012FD4DFECDF08952F9380EDB1DF0F2D34
:10068000CDDF81EDA8DF0894C9DFE1DF2F91089568
:1006900004E0F02EDD27C6E613E05BD00993139546
:1006A000FA94D9F7089504E0F02EDD27C6E613E0AA
:1006B000099147D01395FA94D9F70895222718E0A5
:1006C000069508F42F0D279507951A95D1F70895EB
:1006D000A4E6B0E0B7FFFECF0895EDE158DFA8EE45
:1006E000B3E0B6FC02C0B7FFFCCF089539D0EAE30F
:1006F0004EDFB3FCFECF01E000938C005FDF009182
:100700008C00C5E7C00F98DEBB20F1F7B0FE09C032
:1007100000918C000395053008F001E000938C00F7
:10072000EDCFB3FE04C00CE311E0D6DEE8CFB4FE9B
:1007300004C001E01FEFD0DEE2CFB5FC01C0E6CF80
:1007400015C0E199FECF6FBA1EBB0DBBE29AE19ACC
:100750000895E199FECF6FBA1EBBE09A0DB30895DC
:1007600004E0F02EDD27C6E718E097CF04E0F02E76
:10077000DD27C6E718E09CCFFFFFFFFFFFFFFFFF6D
:102000005050800400010100141E2532FFFFFFFF25
:10201000FFFFFFFFFFFFFFFFFFFFFFFFFFFFFFFFD0
:10202000FFFFFFFFFFFFFFFFFFFFFFFFFFFFFFFFC0
:10203000FFFFFFFFFFFFFFFFFFFFFFFFFFFFFFFFB0
:10204000FFFFFFFFFFFFFFFFFFFFFFFFFFFFFFFFA0
:10205000FFFFFFFFFFFFFFFFFFFFFFFFFFFFFFFF90
:10206000FFFFFFFFFFFFFFFFFFFFFFFFFFFFFFFF80
:10207000FFFFFFFFFFFFFFFFFFFFFFFFFFFFFFFF70
:10208000FFFFFFFFFFFFFFFFFFFFFFFFFFFFFFFF60
:10209000FFFFFFFFFFFFFFFFFFFFFFFFFFFFFFFF50
:1020A000FFFFFFFFFFFFFFFFFFFFFFFFFFFFFFFF40
:1020B000FFFFFFFFFFFFFFFFFFFFFFFFFFFFFFFF30
:1020C000FFFFFFFFFFFFFFFFFFFFFFFFFFFFFFFF20
:1020D000FFFFFFFFFFFFFFFFFFFFFFFFFFFFFFFF10
:1020E000FFFFFFFFFFFFFFFFFFFFFFFFFFFFFFFF00
:1020F000FFFFFFFFFFFFFFFFFFFFFFFFFFFFFFFFF0
:10210000FFFFFFFFFFFFFFFFFFFFFFFFFFFFFFFFDF
:10211000FFFFFFFFFFFFFFFFFFFFFFFFFFFFFFFFCF
:10212000FFFFFFFFFFFFFFFFFFFFFFFFFFFFFFFFBF
:10213000FFFFFFFFFFFFFFFFFFFFFFFFFFFFFFFFAF
:10214000FFFFFFFFFFFFFFFFFFFFFFFFFFFFFFFF9F
:10215000FFFFFFFFFFFFFFFFFFFFFFFFFFFFFFFF8F
:10216000FFFFFFFFFFFFFFFFFFFFFFFFFFFFFFFF7F
:10217000FFFFFFFFFFFFFFFFFFFFFFFFFFFFFFFF6F
:10218000FFFFFFFFFFFFFFFFFFFFFFFFFFFFFFFF5F
:10219000FFFFFFFFFFFFFFFFFFFFFFFFFFFFFFFF4F
:1021A000FFFFFFFFFFFFFFFFFFFFFFFFFFFFFFFF3F
:1021B000FFFFFFFFFFFFFFFFFFFFFFFFFFFFFFFF2F
:1021C000FFFFFFFFFFFFFFFFFFFFFFFFFFFFFFFF1F
:1021D000FFFFFFFFFFFFFFFFFFFFFFFFFFFFFFFF0F
:1021E000FFFFFFFFFFFFFFFFFFFFFFFFFFFFFFFFFF
:1021F000FFFFFFFFFFFFFFFFFFFFFFFFFFFFFFFFEF
:02220000E4C92F
:00000001FF
